:020000040000FA
:020000000528D1
:08000800052883160130810078
:100010003F30850007308900FF308600A030870020
:100020000C3088009F018312003087009B308800CD
:1000300021309000AF011030A800443084008001CE
:10004000840AA80B1F281030A80054308400C20175
:10005000420803178D0046248000840AC20AA80BB8
:1000600028281D21C301AD01BA01A001A101BD01D4
:100070001D300B118207BF28E528D128DC28E8288D
:10008000EF280528052805284B2957295B296A29C7
:100090008C29D229F2299129D52BAD2AAA2A262BDF
:1000A000C52A232A2F2ADE2B322C392C3E2A4E2A0F
:1000B00071287828822A902AEA2BF42B552B932B2F
:1000C000820700340134053400340934003400342C
:1000D00000340D340B1D6A28BC00C83081003C0878
:1000E000392888170730AF00C83081001E306A28D1
:1000F00010211430A80094201430A8009D208B13E8
:10010000AD08031985288714862887102F0A073918
:10011000AF00B72149215D216C21D621F4212F08A0
:10012000033903190D247F28A401A5010330AA0077
:100130004621A220A80B942808000A30A522A80B6B
:100140009D2808000130A722243084002A08A3003B
:10015000A303A3030008840A0006840AA30BAC28A7
:100160008000243084000B1DB328D83081000B118F
:10017000B00ABD1FF3200930AB0000306A281D21F2
:100180000B1DC028D73081000B11BD1BF320AB0B1A
:10019000CA28EA28800D031CCF2801306A280230C3
:1001A0006A2810210B1DD228D73081000B11B00A0C
:1001B000BD1FF32003306A281D210B1DDD28D73019
:1001C00081000B11BD1BF320C728102104306A28C1
:1001D0001D21C728840A0930AB0005306A28102188
:1001E000AA0BB3280800301BB0013D087F3930024C
:1001F00003180A293008BE00BE0C3E0C0F39303EF1
:1002000003178D004624BE000B21BE0B0429F530D8
:1002100081000B1108006E30A300A30B0D2908000C
:100220002A2187118817000000000000000000004C
:10023000000000000000071508002A21071188139C
:1002400000000000000000000000000000000000AE
:1002500087150800051E2F298F018E0108000C1834
:1002600032290800071187110714A301C2010D21CB
:100270000D210D210D210D210D210D210D210D210E
:100280000D21C20B372907100C1008000A30A722D5
:10029000080009306A281D212F08073CB100B10D64
:1002A000B10D310D383981389F000A306A2810218C
:1002B0001F150B306A281D2108001F195D291E0813
:1002C000B200B20CB2130130320202300319B20094
:1002D0000C306A2810210800C2010230AA00023046
:1002E000A8000430AC0008170000000000009921AD
:1002F0004308060503197E2903147F2903100813F8
:1003000000000000A021C20DAC0B7329A80B8A29A4
:1003100010306A280D306A281D2171294208B30067
:100320006F291021AA0B8E294208B400B31FA929F6
:10033000D4290000000000000000000000000800B8
:1003400000000000000000000000000000000000AD
:100350000800B4093408C200C20E0F30B405C2054B
:100360000A30C2080319C029B407C203B129AF0873
:10037000031DBD290314C30DBF290310C30D0800BD
:1003800043080605031DC9294308210503193A1628
:10039000D029430821050319D0294309AD05A1053A
:1003A0000E306A281D210800B401C0293309B500A8
:1003B0003A1AF02943082105031DF0294C302F0774
:1003C0008400203080070F303505031DE929001611
:1003D000F029001AEC29F0290F30350580060012AB
:1003E0000F306A281021080044302F078400B31F03
:1003F000002A4309AD05801FA42A80130008412B61
:10040000B41734080002031D092A3A1E082A452B96
:10041000B12AB2080319152A4309AD05801FA42A81
:100420004309AD050008B400B12ABF01443084007F
:100430000230A800340800020319BF0A840AA80B7E
:100440001A2A16306A281D210430A8003408000238
:100450000319BF0A840AA80B262A17306A2810211C
:100460000230A800340800020319BF0A840AA80B4E
:10047000322ABF08031D802A1B306A281D21443000
:1004800084002F088407801F4A2A00087F39031D33
:100490004A2ABD014309AD051C306A2810215B22A0
:1004A0003408C2000008B40042088000B41FA42A27
:1004B000B2016E22B12AB4135A30340203193A142D
:1004C0005B3034020319BA145C30340203193A1554
:1004D0005D3034020319BA15B4170800B4135A304A
:1004E000340203193A105B3034020319BA105C303D
:1004F000340203193A115D3034020319BA110800AD
:100500001F306A281021443084002F088407000817
:100510007F39031D8C2ABD014308AD0420306A28B1
:100520001D21801B952A0530A52A80130008B400E0
:100530006E22B201B20AB12AFF30A4000030A50039
:100540000330AA00A220282B0530A7229C2AA9004C
:1005500013306A281D2112306A281021A90BA82AFD
:100560000800B413B408031DBF2A3208BD00BD0C37
:10057000331EBC2ABD17BD2ABD130330A42AA52BE8
:10058000B4080319BD2A15306A281D2160303305CF
:10059000C2000319D22A603042020319D22AC21EB5
:1005A000E12A132B3408A400A4133F30A50032081D
:1005B000A600331ADD2AA617DE2AA6130430AA00E5
:1005C000242B3408A400A413A50132030319102B13
:1005D00003303205BE003208B100B10CB10C1F303F
:1005E000B10502303102031C0E2B4C302F07840062
:1005F000000EA300230C03393E02031C082B031931
:10060000082B081D082B1F30B1053102031DB10A4C
:10061000310C03182516A5043423242BB101082B13
:100620003208A5000C2B3408A400A41332030319CC
:100630002F2BB20CB20C320CA50025124C302F0718
:10064000840000182516342314306A281021A220B3
:100650003A1F0800BA1F322B0530A722C22B3208DE
:10066000A500232B3A130800331A382BA516392B73
:10067000A512A51325170330AA000800331E382B36
:10068000362BB400B201B20A6E2235080F39A3002E
:1006900003199C2B0930230203189C2B230860208C
:1006A00003199C2BA30023306A281D21A303C20138
:1006B000AE01AC013408A200A213AC0A2308543ED8
:1006C000840000080319742B7F39220203196B2B55
:1006D000A208031D6D2B2C08AE00AC0A840A05305D
:1006E0002C02031D612B772B2C08C2006D2B0430CC
:1006F00084022E0803197F2B2E038407A02B4208A7
:1007000003199C2B4203840722088000331A8017A8
:10071000000803178C0003135430040203178D00E4
:10072000031324306A201021831603178C130C1531
:100730003B244308A104AD043A120430A722B12A95
:10074000800103178C0103138C2B5A303402031CD5
:10075000D02B033C031CD02BBA173A173308BB002D
:100760005A30B4020310B40DB40D54303407AE0047
:100770000430AC002E0884000008031DC42BAC0B11
:10078000C22BCE2BAE0ABA2BB4003B08B41FC92B28
:10079000103AB300B4130430A722C02ABA13C42BF2
:1007A000BF015430840011306A281D210124003C0F
:1007B0000319DC2B3A18BF0A18306A2810210230BE
:1007C000A722840A0124003C0319E82BBA18BF0AA7
:1007D00021306A281D21840A0124003C0319F22BD0
:1007E0003A19BF0A22306A281021840A0124003CE9
:1007F0000319FC2BBA19BF0ABF080319C02A043019
:10080000A52A0430B70000087F39340203190134E7
:10081000B70B0B2C0034840A032C200A0739A000E4
:10082000A008031D162C0130A8009D20443020078D
:100830008400801F302C0008A400A413A40803190E
:10084000302C4C302007840000080F39A500A50C7F
:1008500003182516A5170330AA004621A220080078
:1008600019306A281D2108308407E03080051A30CD
:100870006A28102108008B1355308D00AA308D0096
:100880008C1400000C1183120313080083168C13C0
:0A0890000C1483120C080313080077
:02400E00723FFF
:1042000000000000000000000000000000000000AE
:10421000000000000000000000000000000000009E
:104260000700080009000A000C000E0010001300EF
:1042700018001D002500300041005D009100FF0086
:00000001FF
